:0400000000000000FC
:0400010000000000FB
:0400020000000000FA
:040003002EC6000005
:0400040014280A2191
:04000500190400AF2B
:0400060000000000F6
:0401000000000000FB
:040101000CC6624086
:0401020015C20725F6
:040103002DAA50A52C
:040104000B0421D1F6
:040105001B8A5625D6
:0401060019285C0157
:040107002F0420F7AA
:040108002DAA50A527
:040109000B0421D1F1
:04010A003B280A0480
:04010B002DC6A2401B
:04010C0000000000EF
:04010D003B280A047D
:04010E00260421CFD3
:04010F0000000000EC
:0402000000000000FA
:040201001EB286A8FB
:04020200328287A815
:0402030020C603E02E
:04020400188A06202E
:04020500030440812D
:0402060031C20740BA
:040207003EB2800083
:040208003EB2800082
:040209002D820740FB
:04020A002150000F70
:04020B002AC6000EF1
:04020C001B82E6AEBD
:04020D0038B226AF2E
:04020E003B20000091
:04020F00003C0000AF
:04021000383800007A
:040211000F04422F65
:0402120000000000E8
:0404000000000000F8
:0404010019C6E240F6
:040402003B280A0485
:0404030035C2078176
:04040400169016A98F
:040405002150000F73
:0404060021C6004EBD
:040407001682E02E4B
:040408002150000F70
:040409002EC7FFE318
:04040A0004C6010F14
:04040B0031B22021C9
:04040C001F8211EF4B
:04040D0008C6000419
:04040E0032C2078966
:04040F003EC207C121
:040410002420120191
:0404110019C2070104
:040412002DA41060A5
:040413000504851146
:0404140007201200AB
:0404150000000000E3
:0404160009E6404172
:0404170039A6106191
:0404180000000000E0
:040419000FE6404268
:04041A0010B280425A
:04041B0010B2804259
:04041C0034AA2022BC
:04041D002820200073
:04041E00133C20006B
:04041F002B38200056
:0404200013824624D9
:040421001088478078
:0404220037884120B6
:040423002D0482D052
:040424000FE640425D
:040425000D0484B787
:040426002F282C004F
:040427000C0486CF6C
:040428001DB3F128E7
:0404290021B380215A
:04042A0027B3802252
:04042B003B7A0041D7
:04042C0032AA2021AF
:04042D000920100092
:04042E00323C10004C
:04042F000A38100077
:0404300013824624C9
:040431001D884100E1
:0404320003048681B8
:0404330003BE0021E3
:0404340037884120A4
:04043500200485B06A
:0404360037C207E0E2
:040437003B20000066
:040438000804871716
:040439002EC60000CB
:04043A0014280A2157
:04043B000704876FBC
:04043C0000000000BC
:0407000010C6E048F7
:040701000A04E0CF37
:040702002BC60240C0
:040703003B280A0481
:040704000104E08F7D
:0407050000000000F0
:0407060002C6004FD8
:04070700005000039B
:040708000328F17958
:0407090023C600E023
:04070A000504E157AA
:04070B000050000397
:04070C002028017828
:04070D000804E1B744
:04070E002150000F67
:04070F0036ECF0E0F4
:040710000D04E217DB
:0407110017E6600285
:0407120004C6008396
:0407130034C6E2A75F
:040714002504E4CF05
:040715001CC6E2E636
:040716001704E9AF2C
:0407170015C6E327F9
:040718001C04E80FC6
:0407190025C60103ED
:04071A0013C6E38798
:04071B002504E4CFFE
:04071C003BC6E3C62F
:04071D001C04E9EFE0
:04071E0013C6E40713
:04071F001C04E80FBF
:040720002C04E417AA
:040721002150000F54
:04072200322840F049
:040723000D04E47766
:040724002B08800F0F
:0407250000000000D0
:040726003DC6E506E1
:040727003E04EB6F32
:0407280011C6E5868B
:0407290013B3F042D4
:04072A001904E9B015
:04072B001C04E9EFD2
:04072C001AC6E5C63E
:04072D001A04E8AF13
:04072E003EC6E606D7
:04072F003304EC0F94
:040730000050000372
:040731003DEC317AF0
:040732002904E65759
:0407330032E660004A
:040734000FB3E0001F
:0407350002A60620F2
:040736003EB270005F
:0407370037B3F08460
:0407380022AA00846D
:0407390012C6E76697
:04073A001104E8EFCF
:04073B003F8A362398
:04073C002104E4C1EF
:04073D003EC6E7E6E7
:04073E003E04EB6F1B
:04073F002B08700F04
:0407400025C6E8469C
:040741003004E96F28
:0407420002C6E8867D
:040743003B04E92F5B
:040744002B08700FFF
:0407450004C60020C6
:040746003804EA2F5A
:0407470009C600C01F
:040748003504EACFBB
:0407490025C6004081
:04074A003804EA2F56
:04074B0028C600A01C
:04074C003504EACFB7
:04074D0002C6008060
:04074E003804EA2F52
:04074F000FC6006071
:040750003504EACFB3
:040751000FAAF00FEC
:040752000050000350
:040753000328F1790D
:040754001004EA970C
:040755001908600F10
:040756002EA6F00FCC
:04075700005000034B
:040758000328F17908
:040759001B04EB375B
:04075A001908600F0B
:04075B0023C600E0D1
:04075C000050000346
:04075D0020280178D7
:04075E001604EBD7BB
:04075F001908600F06
:040760000FC6006060
:040761000050000341
:0407620020280178D2
:040763003C04EC77EF
:040764001908600F01
:040765000000000090
:00000001ff
